:1000000012C02AC029C028C027C026C025C024C0CD
:1000100038C022C021C078C01FC01EC01DC01CC077
:100020001BC01AC019C011241FBECFEDCDBF10E0F8
:10003000A0E6B0E0E0EBF2E002C005900D92A03641
:10004000B107D9F710E0A0E6B0E001C01D92AB36D1
:10005000B107E1F76DD02AC1D3CF20E030E040E016
:1000600050E0A4ECB9E007C0FD013197F1F72F5F34
:100070003F4F4F4F5F4F2617370748075907A0F3E9
:1000800008951F920F920FB60F9211242F938F9302
:100090009F9380E48EB92FB1922F92959F7087B372
:1000A000807F886087BB992321F481E08093610081
:1000B00023C0822F8F70973019F4809362001CC088
:1000C000963021F481E08093600016C0913099F45D
:1000D000813041F487B3807F8A6087BB809166005E
:1000E0008FB90AC08F3019F49093630004C08E302A
:1000F00011F4109263001FB89F918F912F910F9070
:100100000FBE0F901F9018951F920F920FB60F926F
:1001100011248F939F9384B195B19093680080933D
:1001200067009F918F910F900FBE0F901F901895B1
:10013000F89481E0B0D091E09ABB8AE087BB1BBA0B
:100140008BB78BBF85B7816085BF80E888BD18BC41
:1001500085B7806285BF88EF81B910926200909365
:10016000630088E58DB9789481EA90E09093680007
:100170008093670043E0EFEF76E064E05BE8109285
:10018000600046B9809160008823E1F313B8E7B9B5
:1001900080916200833061F0843018F4813069F41A
:1001A00005C0853039F0873041F406C067B905C015
:1001B00077B903C087B901C047B910926100809137
:1001C00061008823E1F356B985B7877E886085BFD3
:1001D0008895809167009091680090936500809366
:1001E000640046B910926100809161008823E1F3B8
:1001F00056B985B7877E886085BF889580916400F1
:10020000909165002091670030916800821B930BEC
:1002100095958795959587958093660098B380917D
:100220006300880F880F880F977F892B88BBA7CF23
:1002300027B3207F922F9A6097BB90E49EB98FB925
:10024000769BFECF286027BB08958A3018F4282FAC
:10025000205D02C0282F295C97B3907F892F8A6088
:1002600087BB80E48EB92FB9769BFECF986097BB91
:1002700008951F93182F82958F70E7DF812F8F705D
:10028000E4DF1F9108951F93182F892FF2DF812F2C
:10029000F0DF1F9108958295880F880F807C886118
:1002A0008DB987B3807F886087BB0895F894FFCFAE
:00000001FF
